:100800008431542CAE3401347E1484314E01961E52
:100810000A2C0B2C122C8C1E0E2C0F2C122CBE31E1
:10082000E92684310B1F152C162C522C4E01991FD2
:100830001A2C1B2C252C8F1F1E2C1F2C252C400105
:100840005C088A005B080A0084314E01191F292CBC
:100850002A2C342C0F1F2D2C2E2C342C40015A08FE
:100860008A0059080A0084314E01991E382C392C0F
:10087000432C8F1E3C2C3D2C432C400158088A00F1
:1008800057080A0084314E01191E472C482C522C5F
:100890000F1E4B2C4C2C522C400156088A00550838
:1008A0000A0084317E10090040018431572CBC318C
:1008B000A1248431E900BC31A2248431EA00410141
:1008C000983100208431EE004201A03100208431B3
:1008D000E50032308400BD308500CC308600013028
:1008E00087000930BC31CB24843145308400BD30D1
:1008F0008500D0308600023087000A30BC31CB241E
:10090000843155308400003085001430BC31C5245A
:10091000843152308400013085001330BC31C5244D
:100920008431A0308400013085001F30BC31C524E3
:10093000843120308400023085005030BC31C52421
:100940008431A0308400023085003030BC31C524B1
:10095000843147308400033085002030BC31C52409
:1009600084317E104001A8319F2841016D080F3E5F
:1009700086000230870001080F39573EE000003042
:1009800003180130E100D22C41016D080F3E8600B2
:100990000230870001080F39303EE00000300318B4
:1009A0000130E1006C086D074201A00020088600BC
:1009B0000230870041016008810001304201A0003F
:1009C00020084101EC0769084201A00041016A08C2
:1009D0004201A100A201A3010830A035A10DA20D82
:1009E000A30D890BED2C41016B084201A400A50168
:1009F000A435A50DA435A50DA435A50DA435A50DCB
:100A0000A435A50D2408103EA6000030253DA70002
:100A10002608A8002708A9000030A91BFF30AA005B
:100A2000AB00200828044101A40042012108290448
:100A30004101A500420122082A044101A600420109
:100A400023082B044101A7006D08A8000230A9006B
:100A50006C084201AC00AD012C084101AA00420122
:100A60002D084101AB00A0310120843141016C0807
:100A70004201A000A10120084101E907420121082B
:100A80004101EA3D5508031D462D472D1E2EFF301E
:100A900042015E05A00000305F05A1000330200682
:100AA0002104031D542D552D1E2E4101EC016C080F
:100AB0006D074201A0002008860002308700323016
:100AC00081000130A00020084101EC076C086D078F
:100AD0004201A00020088600023087000430810017
:100AE0000130A00020084101EC076D086C07A00050
:100AF0000230A1006C30A2000230A3000430A40038
:100B00000030A500B1312621843104304201A0001B
:100B100020084101EC076C086D074201A000200885
:100B2000860002308700363081000130A0002008A6
:100B30004101EC076C086D074201A0002008860007
:100B400002308700043081000130A00020084101FC
:100B5000EC076D086C07A0000230A1006830A2000D
:100B60000230A3000430A4000030A500B1312621DA
:100B7000843104304201A00020084101EC076908DB
:100B80004201A00041016A084201A100A201A301A3
:100B90000830A035A10DA20DA30D890BC92D41016F
:100BA0006B084201A400A501A435A50DA435A50D2F
:100BB000A435A50DA435A50DA435A50D2408103E1A
:100BC000A6000030253DA7002608A8002708A90098
:100BD0000030A91BFF30AA00AB0020082804410107
:100BE000A4004201210829044101A5004201220874
:100BF0002A044101A600420123082B044101A70059
:100C00006D08A8000230A9006C084201AC00AD01DB
:100C10002C084101AA0042012D084101AB00A0317E
:100C20000120843141016C084201A000A10120088B
:100C30004101E907420121084101EA3D4101EC017E
:100C40006C086D074201A000200886000230870072
:100C5000373081000130A00020084101EC0742013B
:100C60006008031D342E352E3B2E02304101E20078
:100C70000030E300402E04304101E2000030E30088
:100C80006C086D074201A000200886000230870032
:100C900041016208810001304201A00020084101A9
:100CA000EC076C086D074201A000200886000230A6
:100CB00087008101810A0130A00020084101EC0772
:100CC0006C086D074201A0002008860002308700F2
:100CD000033081000130A00020084101EC074201EF
:100CE00060080319742E752E942E41016C086D074F
:100CF0004201A00020088600023087003A308100BF
:100D00000130A00020084101EC076C086D0742018A
:100D1000A00020088600023087003B3081000130AF
:100D2000A00020084101EC0741016C086D07420159
:100D3000A0002008860002308700FF3081000130CB
:100D4000A00020084101EC0769084201A000410110
:100D50006A084201A100A201A3010830A035A10D3B
:100D6000A20DA30D890BAE2E41016B084201A40018
:100D7000A501A435A50DA435A50DA435A50DA43553
:100D8000A50DA435A50D2408103EA6000030253D74
:100D9000A7002608A8002708A9000030A91BFF30DB
:100DA000AA00AB00200828044101A4004201210848
:100DB00029044101A500420122082A044101A6009C
:100DC000420123082B044101A7006D08A80002304E
:100DD000A9006C084201AC00AD012C084101AA0039
:100DE00042012D084101AB00A031012084314101B5
:100DF0006C084201A000A10120084101E90742015D
:100E000021084101EA3D6B084201A000A101A03583
:100E1000A10DA035A10DA035A10DA035A10DA035C6
:100E2000A10D2008083EA2000030213DA3002208A9
:100E3000A4002308A5000030A51BFF30A600A700D2
:100E4000003024044101A400243042012504410162
:100E5000A5000030420126044101A60000304201F5
:100E600027044101A7006A08A9006908A800B43155
:100E7000112484314101680803193F2F402F5F2F4F
:100E80000030A000A1000430A2000030A300B03068
:100E9000AA314722843100304101A7000030A6006A
:100EA0000F30A5000030A400B030A8000230A90027
:100EB0000430AA000030AB00A03101208431410190
:100EC0006D08C7000230C8000030C900CA006B08B6
:100ED000A13118218431410168080319702F712F45
:100EE000842F0030A7000030A6000F30A50000308E
:100EF000A4006C30A8000230A9000430AA00003021
:100F0000AB00A0310120843108004001EB00B92F73
:100F100040016B084101B200B301B235B30DB235E7
:100F2000B30DB235B30DB235B30DB235B30D3208D2
:100F3000083EB4000030333DB5003408B600350833
:100F4000B7000030B71BFF30B800B90000303604DE
:100F5000AD0001303704AE0000303804AF0000307F
:100F60003904B0001030B100B0313C20873101307D
:100F7000F72F6B084101B200B301B235B30DB235A2
:100F8000B30DB235B30DB235B30DB235B30D320872
:100F9000083EB4000030333DB5003408B6003508D3
:100FA000B7000030B71BFF30B800B900003036047E
:100FB000A40003303704A50000303804A600003038
:100FC0003904A700A801B3318E2387314101BA004B
:100FD000BB013B08003A0319EE2FF62F3A08003AFE
:100FE0000319B72F1C3A0319882FF62F0030080079
:100FF000E43000320032890BF92F00320032080051
:101000004101A00020084001EB00EB0DEB0D410178
:101010001D0840016B0603396B0641019D001D143C
:1010200008004001EB006B084101B400B501B43584
:10103000B50DB435B50DB435B50DB435B50DB43504
:10104000B50D3408083EB6000030353DB70036080F
:10105000B8003708B9000030B91BFF30BA00BB0038
:1010600000303804A40004303904A50000303A04EC
:10107000A60000303B04A7003308A9003208A800EE
:10108000B4311124883140016B084101B400B5012D
:10109000B435B50DB435B50DB435B50DB435B50DA4
:1010A000B435B50D3408083EB6000030353DB70004
:1010B0003608B8003708B9000030B91BFF30BA0055
:1010C000BB0004303804A40002303904A50000300D
:1010D0003A04A60000303B04A7000A30A800B33150
:1010E0008E23883140016B084101B400B501B4354D
:1010F000B50DB435B50DB435B50DB435B50DB43544
:10110000B50D3408083EB6000030353DB70036084E
:10111000B8003708B9000030B91BFF30BA00BB0077
:1011200000303804AD0001303904AE0000303A041C
:10113000AF0000303B04B0001030B100B0313C20B3
:10114000883140016B084101B400B501B435B50DDB
:10115000B435B50DB435B50DB435B50DB435B50DE3
:101160003408083EB6000030353DB7003608B800F8
:101170003708B9000030B91BFF30BA00BB0004309B
:101180003804A40000303904A50000303A04A60059
:1011900000303B04A700A801A80AB3318E23883190
:1011A00040016B084101B400B501B435B50DB4354B
:1011B000B50DB435B50DB435B50DB435B50D340830
:1011C000083EB6000030353DB7003608B800370895
:1011D000B9000030B91BFF30BA00BB000030380442
:1011E000AD0001303904AE0000303A04AF000030E9
:1011F0003B04B000B101B10AB0313C20883140015C
:101200006B084101B400B501B435B50DB435B50D69
:10121000B435B50DB435B50DB435B50D3408083E4B
:10122000B6000030353DB7003608B8003708B900C1
:101230000030B91BFF30BA00BB0000303804A400F6
:1012400003303904A50000303A04A60000303B0406
:10125000A700A801B3318E238831133A031D312929
:10126000322943280800230843012F06031D48297B
:101270004601220843012E06031D48294601210884
:1012800043012D06031D48294601200843012C0671
:10129000031D4B294C29812946013D08031D512975
:1012A0005229812943012F084101C20043012E0820
:1012B0004101C10043012D084101C00043012C0838
:1012C0004101BF00C301C30A0030A631C6268931DF
:1012D00081294601AE01AE0AA52902302C0746013C
:1012E000A000003043012D3D4601A1000030430124
:1012F0002E3D4601A200003043012F3D4601A300D0
:10130000A52943012F084201C30043012E084201D1
:10131000C20043012D084201C10043012C084201D3
:10132000C00000309E31072689314301BF00C00153
:101330004008003A03199D29A5293F08013A0319DD
:101340006929033A03196D29A5294601440803199F
:10135000AA29AB29B429C40100304101A000A10091
:10136000BF3119278931BE29C401C40A1430410193
:10137000A0000030A100BF31192789310630430198
:10138000C0001330BF00AD30890BC429BF0BC42986
:10139000C00BC429003201304301BF003F084601A1
:1013A000BD0708303D02031CD629D729E129BD011C
:1013B00001304301AC070030AD3D0030AE3D0030A0
:1013C000AF3D00309231E622893146012E080319E3
:1013D000EA29EB293329BE3166268931F7294930BC
:1013E0004101A0002030A100BC31FC248931B5307E
:1013F0004101A0002930A100BD310E2589318B1794
:101400000B174001DF01DF0A00304601B400003055
:10141000B3000030B2000030B10043013C080319B2
:10142000122A132A142C4601C6010030B8000030DD
:10143000B7000030B6000030B5000030BC0000300E
:10144000BB000030BA000030B90046013C083B0444
:101450003A04390403192D2A2E2A562A3C0843013E
:101460002F02031D432A46013B0843012E02031DA0
:10147000432A46013A0843012D02031D432A46012F
:10148000390843012C02031C462A472A562A0030F9
:101490004601BC000030BB000030BA000030B9008B
:1014A0000130B131DE2189314601C60146013808DB
:1014B00037043604350403195E2A5F2AA52A380842
:1014C00043012F02031D742A4601370843012E02EF
:1014D000031D742A4601360843012D02031D742A98
:1014E0004601350843012C02031C772A782AD22AA8
:1014F00000304601B8000030B7000030B6000030C0
:10150000B50046080319852A862A8C2A0130B13194
:10151000DE2189314601C60143012F084101C20085
:1015200043012E084101C10043012D084101C000C3
:1015300043012C084101BF00460141084101C3009D
:101540000030A631C6268931D22A43012F08420134
:10155000C30043012E084201C20043012D0842018D
:10156000C10043012C084201C00000309E31072613
:101570008931023A031DBD2ABE2AD22A0230430114
:101580002C074601B500003043012D3D4601B60051
:10159000003043012E3D4601B700003043012F3D8E
:1015A0004601B80046014608031DD72AD82AF22A68
:1015B0000F304101B2002730B300013088311120D3
:1015C000893100304101A7000030A6002F30A5006E
:1015D0002C30A400A801A80AB3318E23893146011A
:1015E000C601C60A4603031DF62AF72A112B41013C
:1015F000B2010130AB3181238931003A0319012B4B
:10160000022B062B02304601C600112B0130873118
:1016100085278931003A03190E2B0F2B112B460118
:10162000C6010230460146060319172B182B1E2B44
:1016300003304606031D1D2B1E2B2A2B013087313C
:1016400085278931003A0319262B272B2A2B46019F
:10165000C601652B023046014606031D302B312B97
:10166000652B0130B231DE228931003A0319392B62
:101670003A2B562B0130B2310F228931033046010B
:10168000C600013043012C074601B9000030430178
:101690002D3D4601BA00003043012E3D4601BB00FE
:1016A000003043012F3D4601BC00652B0130B231B3
:1016B000742289314101320833040319602B612BF4
:1016C000652BA03149208931652B473043015402F5
:1016D0004601C200420803196E2B6F2BB92B023052
:1016E0004606031D742B752B8A2B47304101C7001A
:1016F0000330C800460142084301BF00C0013F0853
:101700004101C900430140084101CA000130A13133
:10171000182189318B1346014208430154024601C6
:10172000AF0047302F02B00030080319982B992BD7
:10173000B42B47304101A0000330A100460142080C
:10174000473E4101A2000330A30046013008430197
:10175000BF00C0013F084101A4004301400841010E
:10176000A500B1312621893146012F084301D4005B
:101770008B1700309231E622893143014F084E0425
:101780004D044C04031DC52BC62B252A46013408E5
:1017900043012F02031DDC2B4601330843012E02B7
:1017A000031DDC2B4601320843012D02031DDC2BF7
:1017B0004601310843012C02031CDF2BE02B252AB4
:1017C00009303A06031DE52BE62B252A01302C07AC
:1017D000CC0000302D3DCD0000302E3DCE0000303D
:1017E0002F3DCF0004302C074601B10000304301EB
:1017F0002D3D4601B200003043012E3D4601B300AD
:10180000003043012F3D4601B40043015108031944
:101810000A2C0B2C252A0A304101A0000030A1001F
:10182000BF3119278931252A64304101A0003F309A
:10183000A100BD310525893143013E080319212C42
:10184000222C2A2C3B080319262C272C2A2CB431B5
:10185000E624893101309231E622893143014F0873
:101860004E044D044C04031D362C372C842C4601A9
:10187000340843012F02031D4D2C46013308430158
:101880002E02031D4D2C4601320843012D02031D7B
:101890004D2C4601310843012C02031C502C512CC5
:1018A000842C09303A06031D562C572C842C013009
:1018B0002C07CC0000302D3DCD0000302E3DCE0059
:1018C00000302F3DCF0004302C074601B10000301E
:1018D00043012D3D4601B200003043012E3D46013B
:1018E000B300003043012F3D4601B40043015108CD
:1018F00003197B2C7C2C842C0A304101A000003081
:10190000A100BF311927893168304301BF00E4309D
:10191000890B882CBF0B882C00001C2C8431542C84
:1019200064304101A0000230A100A430A2000230C6
:10193000A3000430A4000030A500B13126218C3171
:101940001A2F60304101A0000230A100A430A20093
:101950000230A3000430A4000030A500B1312621DC
:101960008C311A2FFF30A0000030A1000030A200FF
:101970000030A300450124084201A40045012508C8
:101980004201A500450126084201A600450127089D
:101990004201A7001830A736A60CA50CA40C890B91
:1019A000CB2C2408A0052508A1052608A205270898
:1019B000A3050030A800FF30A9000030AA000030C5
:1019C000AB00450124084201AC0045012508420155
:1019D000AD00450126084201AE004501270842013D
:1019E000AF000830AF36AE0CAD0CAC0C890BF22C4E
:1019F0002C08A8052D08A9052E08AA052F08AB0557
:101A00000030B0000030B100FF30B2000030B30051
:101A1000450124084201B400450125084201B500F2
:101A2000450126084201B600450127084201B700DA
:101A30000830B435B50DB60DB70D890B192D340826
:101A4000B0053508B1053608B2053708B3050030D2
:101A5000B8000030B9000030BA00FF30BB004501CB
:101A600024084201BC00450125084201BD00450192
:101A700026084201BE00450127084201BF00183078
:101A8000BC35BD0DBE0DBF0D890B402D3C08B80502
:101A90003D08B9053E08BA053F08BB053808B00443
:101AA0003908B1043A08B2043B08B3043008A8046A
:101AB0003108A9043208AA043308AB04200828041A
:101AC000D60021082904D70022082A04D8002308B8
:101AD0002B04D9001A2F450124084101DB001A2FDD
:101AE00068304101A0000230A100A430A200023001
:101AF000A3000430A4000030A500B13126218C31B0
:101B00001A2FFF30A0000030A1000030A2000030EA
:101B1000A300450124084201A40045012508420113
:101B2000A500450126084201A600450127084201FB
:101B3000A7001830A736A60CA50CA40C890B9A2D6B
:101B40002408A0052508A1052608A2052708A30545
:101B50000030A800FF30A9000030AA000030AB0020
:101B6000450124084201AC00450125084201AD00B1
:101B7000450126084201AE00450127084201AF0099
:101B80000830AF36AE0CAD0CAC0C890BC12D2C0857
:101B9000A8052D08A9052E08AA052F08AB050030B9
:101BA000B0000030B100FF30B2000030B30045019A
:101BB00024084201B400450125084201B500450151
:101BC00026084201B600450127084201B700083047
:101BD000B435B50DB60DB70D890BE82D3408B00539
:101BE0003508B1053608B2053708B3050030B8002E
:101BF0000030B9000030BA00FF30BB0045012408B6
:101C00004201BC00450125084201BD0045012608EE
:101C10004201BE00450127084201BF001830BC3513
:101C2000BD0DBE0DBF0D890B0F2E3C08B8053D083C
:101C3000B9053E08BA053F08BB053808B0043908A5
:101C4000B1043A08B2043B08B3043008A8043108D0
:101C5000A9043208AA043308AB0420082804D200DF
:101C600021082904D30022082A04D40023082B04C5
:101C7000D5001A2FFF30A0000030A1000030A200D4
:101C80000030A300450124084201A40045012508B5
:101C90004201A500450126084201A600450127088A
:101CA0004201A7001830A736A60CA50CA40C890B7E
:101CB000532E2408A0052508A1052608A2052708FB
:101CC000A3050030A800FF30A9000030AA000030B2
:101CD000AB00450124084201AC0045012508420142
:101CE000AD00450126084201AE004501270842012A
:101CF000AF000830AF36AE0CAD0CAC0C890B7A2EB1
:101D00002C08A8052D08A9052E08AA052F08AB0543
:101D10000030B0000030B100FF30B2000030B3003E
:101D2000450124084201B400450125084201B500DF
:101D3000450126084201B600450127084201B700C7
:101D40000830B435B50DB60DB70D890BA12E34088A
:101D5000B0053508B1053608B2053708B3050030BF
:101D6000B8000030B9000030BA00FF30BB004501B8
:101D700024084201BC00450125084201BD0045017F
:101D800026084201BE00450127084201BF00183065
:101D9000BC35BD0DBE0DBF0D890BC82E3C08B80566
:101DA0003D08B9053E08BA053F08BB053808B00430
:101DB0003908B1043A08B2043B08B3043008A80457
:101DC0003108A9043208AA043308AB042008280407
:101DD0004301A8004201210829044301A90042014E
:101DE00022082A044301AA00420123082B044301CC
:101DF000AB001A2F60084201A000A1012108003A9F
:101E00000319032F1A2F2008013A0319902C023AC4
:101E10000319A12C303A0319B22C063A03196B2D81
:101E2000033A0319702D0C3A0319812D013A031955
:101E30003A2E1A2F410163086502031D212F620803
:101E40006402031C242F262FAE31B52E41016408F5
:101E50006202D3006508633BD4006608BD31FE25ED
:101E60008C31FF3042015E05A00000305F05A1000B
:101E7000033020062104031D3E2F3F2FFD2F59085C
:101E8000031D4D2F5808031D4D2F5708031D4D2FBF
:101E9000F030560203184D2F4E2F572F00304201BD
:101EA000D9000030D8000030D700F030D600420111
:101EB0005508031D672F5408031D672F5308031D82
:101EC000672F78305202031C662F672F7A2F42014A
:101ED00059085502031D762F58085402031D762F0A
:101EE00057085302031D762F56085202031C792F00
:101EF0007A2F992F42015608A0005708A1005808D0
:101F0000A2005908A3000330A336A20CA10CA00C18
:101F1000890B842F0230A035A10DA20DA30D890BD2
:101F20008B2F2308D5002208D4002108D3002008D5
:101F3000D20043012B08031DA92F2A08031DA92F36
:101F40002908031DA92FD2302802031CA82FA92F6E
:101F5000C32F4201590843012B02031DBF2F420129
:101F6000580843012A02031DBF2F420157084301AD
:101F70002902031DBF2F4201560843012802031CFA
:101F8000C22FC32FFD2F42015608A0005708A10001
:101F90005808A2005908A3000330A336A20CA10CD4
:101FA000A00C890BCD2F23084101AD00420122086E
:101FB0004101AC00420121084101AB00420120086F
:101FC0004101AA000030B1000030B0000030AF0085
:101FD0000730AE00B23140228C3141012D0843015F
:101FE000AB0041012C084301AA0041012B08430129
:101FF000A90041012A084301A80041015B0808002B
:102000004101A70043013C080319072808285A2862
:1020100065305402031C0D280E281328BE31BD263E
:1020200090310030BC2841016E0803191828192886
:1020300024282703031D1D281E283228803024024F
:10204000031823282428322843015408860003302B
:1020500087004101240881000130A50025084301C3
:10206000D4075828430154088600033087004101F3
:102070002408A5000630A536890B3B282708A600B2
:102080000130A635FF3E031D412826352504C03802
:1020900081000130A50025084301D40754088600BB
:1020A00003308700410124083F39803881002C2803
:1020B0000130BC283E0803195E285F286F283B08C2
:1020C0000319632864286F285008031968286928B1
:1020D000112840018D1C6D286E286F281128BC31F5
:1020E000ED249031003A0319762877287D284201A3
:1020F000630803197C287D2880284E0119160E28B4
:1021000041016E0803198528862898282703031D96
:102110008A288B289D2840016008031D902891285B
:102120009D288030410124020318972898289D2873
:102130002408BD3183259031582841012408A50089
:102140000630A536890BA1282708A6000130A63540
:10215000FF3E031DA72826352504C038BD31832541
:102160009031410124083F3980384201E400E30105
:10217000E30A4E011916582808004101E6006608D6
:10218000B2317422903141013308D8003208D700AF
:10219000003058020830031957020318D028D128FC
:1021A000D428FF308F31FF2FA430C7000230C80081
:1021B0000830C9000030CA006608B531D325903117
:1021C00041014808E5004708E40000306502083096
:1021D000031964020318ED28EE28EF28D1284501E1
:1021E00029084201A000A101450128084201A200DE
:1021F000A3012208A300A201200822044101D90062
:102200004201210823044101DA0045012B08420163
:10221000A000A10145012A084201A200A301220851
:10222000A300A201200822044101E200420121088A
:1022300023044101E300003063022C3003196202E1
:10224000031C232924292B29433059065A04031936
:102250002A292B2934296308D4006208D300660890
:10226000BD31FE259031D128A430C7000230C8000E
:102270002C30C9000030CA006608B531D325903132
:1022800041014808E5004708E400003065022C30B1
:102290000319640203184D294E2959296408620262
:1022A000D3006508633BD4006608BD31FE2590313C
:1022B000D12802304501240603195F2960296C29C1
:1022C000410164086202D3006508633BD4006608DC
:1022D000BD31FE259031D128FF304201A0000030F1
:1022E000A1000030A2000030A300450128084201EF
:1022F000A400450129084201A50045012A08420120
:10230000A60045012B084201A7001830A736A60CED
:10231000A50CA40C890B86292408A0052508A10575
:102320002608A2052708A3050030A800FF30A90051
:102330000030AA000030AB00450128084201AC0083
:10234000450129084201AD0045012A084201AE00BD
:1023500045012B084201AF000830AF36AE0CAD0C82
:10236000AC0C890BAD292C08A8052D08A9052E0851
:10237000AA052F08AB050030B0000030B100FF30D7
:10238000B2000030B300450128084201B400450105
:1023900029084201B50045012A084201B60045015D
:1023A0002B084201B7000830B435B50DB60DB70D96
:1023B000890BD4293408B0053508B1053608B205B3
:1023C0003708B3050030B8000030B9000030BA005B
:1023D000FF30BB00450128084201BC004501290827
:1023E0004201BD0045012A084201BE0045012B08FB
:1023F0004201BF001830BC35BD0DBE0DBF0D890BAD
:10240000FB293C08B8053D08B9053E08BA053F0858
:10241000BB053808B0043908B1043A08B2043B08D7
:10242000B3043008A8043108A9043208AA04330808
:10243000AB04200828044101DC00420121082904E2
:102440004101DD00420122082A044101DE0042016F
:1024500023082B044101DF004401550841015F02BC
:10246000031D422A4401540841015E02031D422A11
:102470004401530841015D02031D422A44015208F0
:1024800041015C02031C452A462A5F2A5F0842017B
:102490005D02031D5B2A41015E0842015C02031DCF
:1024A0005B2A41015D0842015B02031D5B2A410179
:1024B0005C0842015A0203185E2A5F2A6B2A410116
:1024C00064086202D3006508633BD4006608BD312E
:1024D000FE259031D1284101560886000130870041
:1024E0005C08C03F5D08C13F5E08C23F5F08C33F54
:1024F0000030A7000030A6000930A5000030A4007D
:10250000C630A8000230A9000630AA000030AB0097
:10251000B43155249031C6304101A0000630A100ED
:102520000030A200C030B331CE23903141012008E9
:10253000210403199C2A9D2AA82A64086202D30058
:102540006508633BD4006608BD31FE259031D12873
:10255000420160080319AD2AAE2ABE2A6C3041013F
:10256000A0000230A100B430A2000230A300043069
:10257000A4000030A500B13126219031C0304101C6
:10258000D3000030D4006608BD31FE2590314101F2
:102590005308E4075408E53DA430C7000230C800E2
:1025A0000430C9000030CA006608B531D325903127
:1025B00041014708E4074808E53D6330450124062A
:1025C000031DE42AAE316C2EAE317E2E4101E400B3
:1025D00040010E1FEC2AED2AF12A8D1BF02AF12A68
:1025E000002B420161080319F62AF72AFA2ABE31A4
:1025F000D32692314201E101E10A4101E401E40AFA
:1026000043013C080319052B062B092BB4319C24EC
:10261000923142016108031D0E2B0F2B2C2D41011D
:102620006E080319142B152B2C2DE901E90AA12C96
:102630004401BE01BE0A01304101D8005808E90733
:1026400069083D3E8600023087008101810A013021
:10265000D8005808E9070030BF314B2792314101BB
:102660002108E8002008E70069083D3E86000230A6
:102670008700680881000130D8005808E907690818
:102680003D3E860002308700670881000130D80097
:102690005808E9076E0803194E2B4F2B552B4301A1
:1026A0005308031D542B552B592B4101DA01DB0133
:1026B0005E2B02304101DA000030DB0043013C08B0
:1026C000031D632B642B682B4101DC01DD016D2BA5
:1026D00004304101DC000030DD0043013B08031DF4
:1026E000722B732B772B4101DE01DF017C2B08302D
:1026F0004101DE000030DF0043013E08031D812B55
:10270000822B882B10304101E0000030E1008B2B40
:102710004101E001E10143013D08031D902B912B94
:10272000952B4101E201E3019A2B20304101E200A7
:102730000030E30069083D3E8600023087006E08E5
:10274000031DA32BA52B0130A62B003062046004CF
:102750005E045C045A0481000130D8005808E9077F
:1027600069083D3E86000230870040012308810051
:1027700001304101D8005808E9070130BF314B272B
:10278000923141012108E8002008E70069083D3E38
:102790008600023087006808810001304101D800BE
:1027A0005808E90769083D3E86000230870067083F
:1027B000810001304101D8005808E907C22C0030DF
:1027C000A0000130A1000130A200B131AE21923150
:1027D0004101E501B0311A20923141012108E800A0
:1027E0002008E70069083D3E860002308700670840
:1027F00081000130D8005808E9070130D800580896
:10280000E50709306502031C062C072CEA2BC22CB5
:102810000030A0000030A1000130A200B131AE2193
:1028200092314101E601B0311A2092314101210873
:10283000E8002008E70069083D3E86000230870076
:10284000680881000130D8005808E90769083D3E52
:10285000860002308700670881000130D8005808E0
:10286000E9070230D8005808E60708306602031C62
:102870003A2C3B2C132CC22CAA31E122923141017B
:102880004508E8004408E70068084401BE00CD2B75
:10289000A9312421923141014508E8004408E700AC
:1028A000442CAF313427923141014508E8004408F7
:1028B000E700442C430134083504031D602C612CCF
:1028C000732C4401BE0101304101D8005808E907CA
:1028D00069083D3E86000230870081010130D80042
:1028E0005808E907C22CB51F762C772C802CFF30B6
:1028F0004401BE0001304101D8005808E907842C8A
:1029000034084401BE007A2C013040012802003016
:1029100003192702031C8D2C8E2C972C410169086A
:102920003D3E860002308700FF308100D92B4101F7
:1029300069083D3E8600023087004001270881007B
:10294000D92B400169084101D800D9015908003A42
:102950000319AB2CC22C5808003A0319182B013A62
:102960000319DF2B033A0319082C013A03193C2CF5
:10297000073A0319482C013A0319512C033A031959
:102980005A2CC22CFF304001E9000230410169029B
:10299000031CCB2CCC2C2C2D4201E20141016908F7
:1029A000FF3E4401BD0043013C080319D82CD92C3B
:1029B000F72CF02C420162083D3E86000230870071
:1029C00001084101A4000330903100209231013010
:1029D0004101D80058084201E20701304101E902F3
:1029E00041016908031DF52CF62CDA2C182D410144
:1029F00069084001DD008B13420162083D3E8600FC
:102A00000230870001084101A4000330903100200A
:102A10009231003A03190D2D0E2D172D0130410171
:102A2000D80058084201E20701304001DD028B174F
:102A30004101640803191D2D1E2D3E2D0230410158
:102A4000D9000430D800BA30890B242DD80B242D9E
:102A5000D90B242D00003E2D410164080319312DAE
:102A6000322D3E2D05304101D9000F30D800F13014
:102A7000890B382DD80B382DD90B382D0800982DFF
:102A8000410169084201A00041016A084201A10018
:102A9000A201A3010830A035A10DA20DA30D890B41
:102AA0004B2D41016B084201A400A501A435A50DE1
:102AB000A435A50DA435A50DA435A50DA435A50DEA
:102AC0002408103EA6000030253DA7002608A800D7
:102AD0002708A9000030A91BFF30AA00AB0020087E
:102AE00028044101A4004201210829044101A50054
:102AF000420122082A044101A600420123082B04B6
:102B00004101A7006D08A8000230A9002030AA00EA
:102B10000030AB00A0310120953120304101E907A0
:102B20000030EA3D0130E6070030E73D9D31F62DEB
:102B30004101EC016C086D074201A00020088600ED
:102B400002308700633081000130A000200841017D
:102B5000EC076C086D074201A000200886000230D7
:102B60008700823081000130A00020084101EC077D
:102B70006C086D074201A000200886000230870023
:102B8000533081000130A00020084101EC076C089F
:102B90006D074201A00020088600023087006330E4
:102BA00081000130A00020084101EC076C086D078E
:102BB0004201A000200886000230870035308100E5
:102BC0000130A00020084101EC076C086D074201AC
:102BD000A00020088600023087008101810A0130B0
:102BE000A00020084101EC076C086D074201A0001D
:102BF00020088600023087005E0881000130A000B6
:102C000020084101EC076C086D074201A000200874
:102C10008600023087003D3081000130A00020088E
:102C20004101EC076C086D074201A00020088600F6
:102C300002308700073081000130A00020084101E8
:102C4000EC076C086D074201A000200886000230E6
:102C500087008101810A0130A00020084101EC07B2
:102C60000030A7000030A6000930A5000030A40005
:102C70006D086C07A8000230A9000630AA000030D9
:102C8000AB00B4315524953106304201A000200834
:102C90004101EC076C086D074201A0002008860086
:102CA000023087000C3081000130A0002008410173
:102CB000EC076C086D074201A00020088600023076
:102CC000870020304101A000B830A100B0310020C1
:102CD000953141012008063E810001304201A000EB
:102CE00020084101EC072030A000B830A1006D0899
:102CF0006C07BF31BF27953120304101A000B830AB
:102D0000A100B03100209531410120084201A0000E
:102D100020084101EC076D080D3E86000230870057
:102D200001084201A0000430A036890B942E0A301D
:102D30002002031C9C2E9D2EB32E41016D080D3EDA
:102D400086000230870001084201A0000430A0364E
:102D5000890BA72E2008573E4101D60000300318EA
:102D60000130D700C82E41016D080D3E86000230AB
:102D7000870001084201A0000430A036890BBD2E57
:102D80002008303E4101D600003003180130D70042
:102D90006C086D074201A000200886000230870001
:102DA00041015608810001304201A0002008410184
:102DB000EC076D080D3E8600023087000F300105DC
:102DC0004201A0000A302002031CE72EE82EF72E55
:102DD00041016D080D3E86000230870001080F3961
:102DE000573ED800003003180130D900052F4101AB
:102DF0006D080D3E86000230870001080F39303E15
:102E0000D800003003180130D9006C086D0742016A
:102E1000A000200886000230870041015808810088
:102E200001304201A00020084101EC076D080E3E70
:102E300086000230870001084201A0000430A0365D
:102E4000890B1F2F0A302002031C272F282F3E2F0B
:102E500041016D080E3E86000230870001084201E4
:102E6000A0000430A036890B322F2008573E4101C4
:102E7000DA00003003180130DB00532F41016D08E8
:102E80000E3E86000230870001084201A000043097
:102E9000A036890B482F2008303E4101DA0000306F
:102EA00003180130DB006C086D074201A000200808
:102EB00086000230870041015A088100013042013A
:102EC000A00020084101EC076D080E3E860002308C
:102ED00087000F3001054201A0000A302002031CC8
:102EE000722F732F822F41016D080E3E8600023033
:102EF000870001080F39573EDC000030031801300D
:102F0000DD00902F41016D080E3E860002308700E3
:102F100001080F39303EDC00003003180130DD00BD
:102F20006C086D074201A00020088600023087006F
:102F300041015C08810001304201A00020084101EC
:102F4000EC076D080F3E8600023087000108420141
:102F5000A0000430A036890BAA2F0A302002031CDF
:102F6000B22FB32FC92F41016D080F3E86000230EA
:102F7000870001084201A0000430A036890BBD2F54
:102F80002008573E4101DE00003003180130DF0009
:102F9000DE2F41016D080F3E8600023087000108D8
:102FA0004201A0000430A036890BD32F2008303E08
:102FB0004101DE00003003180130DF006C086D07AE
:102FC0004201A000200886000230870041015E080F
:102FD000810001304201A00020084101EC076D088A
:102FE0000F3E8600023087000F3001054201A0002D
:102FF0000A302002031CFE2F8431B52C8431C42CEE
:103000000134B41A042805280A280530B400003019
:10301000B500642800303405BF0003303505C0001A
:103020003F0840040319152816281B280630B40051
:103030000030B500642834181E281F2824280730C3
:10304000B4000030B5006428B5176428023041018F
:10305000A7000030A8000030A900BD31C325983179
:10306000410128084601BF00410127084601BE0072
:10307000AB303E06343003193F06031D402841287B
:103080006428B0311A209831410121084601BF005F
:10309000410120084601BE003F084301C00046012F
:1030A0003E084301BF004008BF00C00134303F0666
:1030B0004004031D5C285D286428AB304001A20059
:1030C00046013E084001A300BF31802798315401DA
:1030D0001F16B6312626983109304301C0001E3034
:1030E000BF00E430890B7228BF0B7228C00B722816
:1030F0000000003040010E1901304101EE000310C4
:1031000040010E1E03140030031801304301BC00BF
:10311000003040010C1B01304301BE003E08031982
:1031200092289328B0284601AC0141016E0803198A
:103130009A289B28A32840018E1A9F28A028A328FC
:103140004601AC01AC0A46012C08031DA828AA2898
:103150000130AB2800304301D3004001181712138F
:103160004601A601A70100304101A0000130A100E5
:103170000130A200B131AE2198314601C0010930C1
:103180004002031CC428C528C628F4284018C928B2
:10319000CA28CD28A801A901D1280830A8000030EC
:1031A000A900B0311A209831FF30410120054301B8
:1031B000BF000030410121054301C0004601280A3B
:1031C0004301E428BF35C00D890BE2283F084601C2
:1031D000A606430140084601A70601304301BF008F
:1031E0003F084601C007BF2827084101A10046014A
:1031F00026084101A000BD317625983143013C08E5
:10320000031D0429A8311B28A83143284001EB00E5
:103210006B084101B700B801B735B80DB735B80D27
:10322000B735B80DB735B80DB735B80D3708083E06
:10323000B9000030383DBA003908BB003A08BC007C
:103240000030BC1BFF30BD00BE0000303B04A400BA
:1032500004303C04A50000303D04A60000303E04CC
:10326000A7003308A9003208A800B431112499310D
:1032700040016B084101B700B801B735B80DB7354B
:10328000B80DB735B80DB735B80DB735B80D370827
:10329000083EB9000030383DBA003908BB003A0892
:1032A000BC000030BC1BFF30BD00BE0000303B0442
:1032B000A4000C303C04A50000303D04A600003002
:1032C0003E04A7003408A8000230A9000430AA0078
:1032D0000030AB00A0310120993140016B08410161
:1032E000B700B801B735B80DB735B80DB735B80D5B
:1032F000B735B80DB735B80D3708083EB9000030FE
:10330000383DBA003908BB003A08BC000030BC1B8D
:10331000FF30BD00BE0000303B04A40010303C0470
:10332000A50000303D04A60000303E04A70036088A
:10333000A9003508A800B4311124993140016B0867
:103340004101B700B801B735B80DB735B80DB7357D
:10335000B80DB735B80DB735B80D3708083EB90008
:103360000030383DBA003908BB003A08BC000030D4
:10337000BC1BFF30BD00BE0000303B04AD0001307F
:103380003C04AE0000303D04AF0000303E04B0000D
:103390001030B100B0313C20993140016B0841013F
:1033A000B700B801B735B80DB735B80DB735B80D9A
:1033B000B735B80DB735B80D3708083EB90000303D
:1033C000383DBA003908BB003A08BC000030BC1BCD
:1033D000FF30BD00BE0004303B04A40000303C04BC
:1033E000A50000303D04A60000303E04A7000230D6
:1033F000A800B3318E23993140016B084101B70019
:10340000B801B735B80DB735B80DB735B80DB73504
:10341000B80DB735B80D3708083EB9000030383D53
:10342000BA003908BB003A08BC000030BC1BFF30B2
:10343000BD00BE0000303B04AD0001303C04AE00D6
:1034400000303D04AF0000303E04B000B101B10ACD
:10345000B0313C20993140016B084101B700B801FF
:10346000B735B80DB735B80DB735B80DB735B80D98
:10347000B735B80D3708083EB9000030383DBA00FE
:103480003908BB003A08BC000030BC1BFF30BD004F
:10349000BE0000303B04A40003303C04A500003013
:1034A0003D04A60000303E04A700A801B3318E23DE
:1034B0009931223A031D5D2A5E2A9E290800D030E8
:1034C000860002308700B43084000030850006306A
:1034D0004101B00016001A00B00B6A2A0030CF007C
:1034E0000030CE000030CD000030CC00450159083E
:1034F0004101C700450158084101C6004501570870
:103500004101C500450156084101C4003F30D200C9
:103510000030A0000030A1000130A200B131AE2186
:103520009A314101C901C90AD301D701B0311A202A
:103530009A3141012108D1002008D0005708031D0D
:10354000A22AA32AB02A5108C800C81AA82AAA2A5F
:103550000130AB2A0030C90048081F39D300B92A0E
:1035600003305706031DB52AB62AB92A51083F3938
:10357000D2005708CC3E86008701500881005708CA
:103580000319C32AC42AD02A4908031DC82AC92AF4
:10359000D02A5708023EB43E8600870150088100B9
:1035A0000130B0003008D70704305702031CD92A75
:1035B000DA2A962A49080319DE2ADF2A032B063065
:1035C000A0000130A1000130A200B131AE219A313A
:1035D0004101CB01B0311A209A3141012108BB00D1
:1035E0002008BA004B08033EB43E860087013A0823
:1035F00081000130B0003008CB0703304B02031CC0
:10360000022B032BEA2A0030A7000030A600093065
:10361000A5000030A400B430A8000030A900063096
:10362000AA000030AB00A03101209A311F304101C7
:10363000530603191C2B1D2B252B4D084E044F043C
:103640004C04031D242B252B272B0130132C003079
:10365000A7000030A6000F30A5000030A400CC3039
:10366000A8000030A9000430AA000030AB00A0314F
:1036700001209A314101D5015308D6000830560285
:103680000318432B442B692B56080319482B492B4D
:10369000622B0130B0000030B1005608083C890AA6
:1036A000532BB035B10D890B512B3008FF3EB200C2
:1036B000FF30313DB300FF303206BE00003033062C
:1036C000BF00642BBE01BF013F08BD003E08BC0027
:1036D0006D2BFF30BC000030BD005508C43E860095
:1036E00087013C0881005508C43E86008701010817
:1036F000B0005508CC3E86008701300881050130B6
:10370000B0003008D507083056020318882B892BE3
:10371000912B5608B000B1013008C0003108C1003B
:10372000952B0830C0000030C1004008D60204309C
:103730005502031C9C2B9D2B3E2B0030A700003014
:10374000A6000530A5000030A400C430A800003059
:10375000A9000430AA000030AB00A03101209A314A
:103760003F3041015206031DB62BB72BB92B4F1426
:10377000FF2BD21EBC2BBD2BFA2B1F305205B000E5
:1037800047091F3A3004B1003108CF041830530202
:103790000318CB2BCC2BFF2BD4015308CA005408A1
:1037A000C43E860087010109B0005408CC3E860063
:1037B0008701300881040130B0003008D407083098
:1037C0004A020318E42BE52BED2B4A08B000B101A7
:1037D0003008C2003108C300F12B0830C2000030AD
:1037E000C3004208CA0203305402031CF82BF92B11
:1037F000CF2BFF2B52081F39B0003008CF04003008
:10380000A7000030A6000130A5000030A400CC3095
:10381000A8000030A9000430AA000030AB00A0319D
:1038200001209A31003008004101EB006B08420191
:10383000A000A101A035A10DA035A10DA035A10DBD
:10384000A035A10DA035A10D2008083EA200003032
:10385000213DA3002208A4002308A5000030A51BD9
:10386000FF30A600A700003024044101A40024304A
:10387000420125044101A500003042012604410116
:10388000A6000030420127044101A700B731952767
:103890009C3141012508EA002408E900A430ED002C
:1038A0000030A000A1002C30A2000030A3006D0861
:1038B000AA3147229C314501A401A40AA501A50A09
:1038C0000630A600A701FF304201A0000030A10091
:1038D0000030A2000030A3005A08A4005B08A50035
:1038E0005C08A6005D08A7001830A736A60CA50C3A
:1038F000A40C890B752C2408A0052508A105260811
:10390000A2052708A3050030A800FF30A900003059
:10391000AA000030AB005A08AC005B08AD005C08A0
:10392000AE005D08AF000830AF36AE0CAD0CAC0C8D
:10393000890B942C2C08A8052D08A9052E08AA058A
:103940002F08AB050030B0000030B100FF30B200EE
:103950000030B3005A08B4005B08B5005C08B6003C
:103960005D08B7000830B435B50DB60DB70D890B3D
:10397000B32C3408B0053508B1053608B205370850
:10398000B3050030B8000030B9000030BA00FF3095
:10399000BB005A08BC005B08BD005C08BE005D08A7
:1039A000BF001830BC35BD0DBE0DBF0D890BD22C2C
:1039B0003C08B8053D08B9053E08BA053F08BB05F7
:1039C0003808B0043908B1043A08B2043B08B3041B
:1039D0003008A8043108A9043208AA043308AB044B
:1039E000200828044501A8004201210829044501B6
:1039F000A900420122082A044501AA004201230825
:103A00002B044501AB004101E4014401510850047D
:103A10004F044E0403190D2D0E2D212D4201550882
:103A2000031D1D2D5408031D1D2D5308031D1D2DA1
:103A30003C30520203181D2D1E2D212D4101E401A1
:103A4000E40A41016408031D262D282D0130292D8B
:103A50000030D500E501E50A4401510850044F0447
:103A60004E040319342D352D452D43012B08031D1C
:103A7000452D2A08031D452D2908031D452D3C30E1
:103A80002802031C442D452D542DFF3042015E05B4
:103A9000A00000305F05A100200321040319512D6F
:103AA000522D542D4101E50141016508031D592D99
:103AB0005B2D01305C2D0030E800420160080319E5
:103AC000622D632D672DDF1C662D672D7D2DB03097
:103AD0004101A0000230A1006C30A2000230A3001E
:103AE0000430A4000030A500B13126219C314101F1
:103AF000680803197C2D7D2D822D80304501AE0094
:103B00000030AF0000304101A7000030A6000930AE
:103B1000A5000030A400C030A8000230A900063083
:103B2000AA000030AB00B43155249C314101690832
:103B30004201A00041016A084201A100A201A301C3
:103B40000830A035A10DA20DA30D890BA12D4101B7
:103B50006B084201A400A501A435A50DA435A50D4F
:103B6000A435A50DA435A50DA435A50D2408103E3A
:103B7000A6000030253DA7002608A8002708A900B8
:103B80000030A91BFF30AA00AB0020082804410127
:103B9000A4004201210829044101A5004201220894
:103BA0002A044101A600420123082B044101A70079
:103BB0006D08A8000230A9002C30AA000030AB002C
:103BC000A03101209C312C304101E9070030EA3D51
:103BD0000030A000A1002030A2000030A3006D083A
:103BE000AA3147229C314101E601E7016708803A8A
:103BF0004201A00080302002031D012E0630410149
:103C00006602031C052E95313F2D9531402D420152
:103C1000CC0000304101A7000030A6002E30A500E6
:103C20000030A400A801B3318E239E310139031D59
:103C30001A2E1B2E1D2E0230FF2F430127082604AB
:103C4000250424040319252E262EB52E270842010B
:103C50004302031D3B2E4301260842014202031D7D
:103C60003B2E4301250842014102031D3B2E430127
:103C7000240842014002031C3E2E3F2EB52E600850
:103C80000319432E442EB02E00304301330240303E
:103C900003193202031C4D2E4E2EB02E023042016B
:103CA0005E06031D572E5F03031D572E582E632EED
:103CB00000304301A7000030A6000030A50000300E
:103CC000A4000230FF2F03305E06033003195F06A5
:103CD00003196B2E6C2E6D2E582E5908031D7B2E4A
:103CE0005808031D7B2E5708031D7B2E3C305602BF
:103CF00003187B2E7C2E7D2E582E01304201D536A6
:103D0000D40CD30CD20C890B7E2E01304301AB3680
:103D1000AA0CA90CA80C890B862E01304201D936B9
:103D2000D80CD70CD60C890B8E2E40085207C40035
:103D30004108533DC5004208543DC6004308553D67
:103D4000C70047084401D100420146084401D000A1
:103D5000420145084401CF00420144084401CE001D
:103D6000FF304201DE05FE30DF0542015F18B92E4B
:103D7000BA2EEC2E4C089C3114249E3142015F1463
:103D80004008C4004108C5004208C6004308C700F7
:103D9000430132084201C800430133084201C9000F
:103DA000CA01CB014808C4074908C53D4A08C63DB9
:103DB0004B08C73D47084301A7004201460843019D
:103DC000A600420145084301A50042014408430101
:103DD000A400BD31EA259E3142015D08D0005C0897
:103DE000CF005B08CE005A08CD004D304101D6000F
:103DF00042014C089031BD209E314201D100510A50
:103E0000031D032F042FE62FFF30FF2F0230510632
:103E1000031D0B2F0C2F192F5008DD004F08DC005D
:103E20004E08DB004D08DA000330DE000030DF0012
:103E3000FE2F0130DE000030DF00FE2F053051067E
:103E4000031D232F242FB82F5008DD004F08DC005E
:103E50004E08DB004D08DA0000304101A7000030B9
:103E6000A6000F30A5000030A4006C30A80002307E
:103E7000A9000430AA000030AB00A03101209E311F
:103E800000304101A7000030A6000530A500003039
:103E9000A4006430A8000230A9000430AA00003059
:103EA000AB00A03101209E3100304101A70000305D
:103EB000A6000130A5000030A4006030A800023048
:103EC000A9000430AA000030AB00A03101209E31CF
:103ED000420143084301A700420142084301A600F2
:103EE000420141084301A500420140084301A400EA
:103EF00042015508031D872F5408031D872F5308BF
:103F0000031D872F3C3052020318872F882F922FD2
:103F10003C304301A4070030A53D0030A63D0030F1
:103F2000A73DA22F420152084301A40742015308B2
:103F30004301A53D420154084301A63D42015508F5
:103F40004301A73D27084401D1004301260844014D
:103F5000D000430125084401CF0043012408440157
:103F6000CE0003304201DE000330DF000130FF2FBE
:103F700006305106031DBD2FBE2FBF2F192F033052
:103F8000DE000030DF00FE2F05305106031DC92F73
:103F9000CA2FFE2F5008DD004F08DC004E08DB0062
:103FA0004D08DA003C3040074301A40000304201D4
:103FB000413D4301A50000304201423D4301A600BE
:103FC00000304201433D4301A700FE2F5F08013A44
:103FD0000319EE2F023A0319F92FFE2F5E08013A5A
:103FE0000319062F023A03191E2F0B3A0319C42F87
:103FF000FE2F5E08033A03191E2FFE2F0030080023
:1040000001344001991241012408AC002508AD009B
:104010002608AE002708AF001030AF36AE0CAD0C4E
:10402000AC0C890B0D282C084001E4004101240848
:10403000AC002508AD002608AE002708AF00083008
:10404000AF36AE0CAD0CAC0C890B20282C0840010F
:10405000E5004101240804384001E60064304101D4
:10406000A0000030A1000330A2000030A300B03156
:10407000FD20A03141012908A1002808A0002B083B
:10408000A3002A08A200BF31DF27A0314001991602
:1040900008007E1C4D28AC31E62C4101D6014301BD
:1040A0003C080319542855286A28D7304101C70015
:1040B0000030C8000130C9000030CA000130B531FD
:1040C000D325A03141014703480403196828692812
:1040D0008128172942011D1D6E286F287128400173
:1040E0005E1642019D1C752876287D281D121D161E
:1040F0004001DE164101D601D60A420119084101EC
:10410000D70056080319852886288A28BE31BD267F
:10411000A03117296E08031D8E288F2806295708FD
:10412000A8310020A0311729400163084101D300C4
:104130000230D336890B992853080F39D5003F3008
:104140005705D3004001630803394101D40005300D
:10415000D435FF3E031DA82854355304D700D82872
:1041600057084001EA00E301E201DF01DF0AEE281F
:104170005708A8310020A031EE2857084001E1007F
:10418000AA306106031DC528C628C828E201EE280A
:10419000E201E20A01304101A0000030A100BF317C
:1041A0001927A031EE2857084001E900DD01EE286B
:1041B0005508D300D4015408003A0319E028EE282A
:1041C0005308003A0319B028013A0319B828033AF2
:1041D0000319BD28013A0319D328EE284001E30151
:1041E000172957084001E300172940016008031907
:1041F000FA28FB2800295E16BE31BD26A031EE2824
:1042000041015708A8310020A031EE285708C039D5
:10421000D300D4015408003A03190F29F528530894
:10422000803A03199428403A0319F128F528080028
:104230004101D40049084A0403191F2920293229C1
:104240004808B3004708B2004A08B5004908B4005E
:104250005408A231CF22A131003A031D302931295F
:104260003229F22941015408CB00CC01CB35CC0DC9
:10427000CB35CC0DCB35CC0DCB35CC0DCB35CC0DDA
:104280004B08083ECD0000304C3DCE004D08CF001D
:104290004E08D0000030D01BFF30D100D2000030DB
:1042A0004F04AD0001305004AE0000305104AF00A7
:1042B00000305204B0002030B100B0313C20A131B8
:1042C00041015408CB00CC01CB35CC0DCB35CC0D06
:1042D000CB35CC0DCB35CC0DCB35CC0D4B08083EBA
:1042E000CD0000304C3DCE004D08CF004E08D00030
:1042F0000030D01BFF30D100D20000304F04A400AA
:1043000002305004A50000305104A60000305204D1
:10431000A700A801B3318E23A1314101D300531E60
:1043200092299329C1295408CB00CC01CB35CC0D5F
:10433000CB35CC0DCB35CC0DCB35CC0DCB35CC0D19
:104340004B08083ECD0000304C3DCE004D08CF005C
:104350004E08D0000030D01BFF30D100D200043016
:104360004F04A40002305004A50000305104A60000
:1043700000305204A7001830A800B3318E23A131B9
:10438000F229D31DC429C52960295408CB00CC01CA
:10439000CB35CC0DCB35CC0DCB35CC0DCB35CC0DB9
:1043A000CB35CC0D4B08083ECD0000304C3DCE0047
:1043B0004D08CF004E08D0000030D01BFF30D10098
:1043C000D20004304F04A40002305004A500003095
:1043D0005104A60000305204A7000830A800B331F1
:1043E0008E23A13108004601C4010530AA00003027
:1043F000AB0000304101A7000030A6003930A50015
:104400000030A400A801B3318E23A1314601A500DC
:104410000430250603190D2A0E2A4C2A44080319D4
:10442000122A132A1C2AC40100304101A000A10055
:10443000BF311927A131262AC401C40A1430410111
:10444000A0000030A100BF311927A1310B3043017A
:10445000C0002630BF005D30890B2C2ABF0B2C2AF0
:10446000C00B2C2A003200309231E622A1310130FB
:104470004601AA020030AB3B2A0A031D432A2B0A3D
:10448000031D432A442AF9290530AA000030AB0055
:10449000B7313527A131F9299A315F22A13146017F
:1044A000C10000304101A7000030A6001930A5006E
:1044B0000430A4000430A800B3318E23A131892A2E
:1044C000460144080319652A662A6F2AC401003090
:1044D0004101A000A100BF311927A131792AC401EF
:1044E000C40A14304101A0000030A100BF311927D7
:1044F000A13103304301C0000830BF007730890B81
:104500007F2ABF0B7F2AC00B7F2A00309231E62220
:10451000A13100304101A7000030A6002E30A500D7
:104520000030A400A801B3318E23A1310139031951
:104530009A2A9B2A602A43012F084101C2004301A5
:104540002E084101C10043012D084101C000430173
:104550002C084101BF00460141084101C300003061
:10456000A631C626A131460141080319B82ABA2A44
:104570008931EB2943012F084601A30043012E088E
:104580004601A20043012D084601A10043012C0869
:104590004601A000BD01BD0AAE018931E5294101F6
:1045A000C60034083504031DD62AD72AD92A01307B
:1045B000BA2B4608B600B701B635B70DB635B70DFC
:1045C000B635B70DB635B70DB635B70D3608083E5A
:1045D000B8000030373DB9003808BA003908BB00D0
:1045E0000030BB1BFF30BC00BD0000303A04A4000B
:1045F00020303B04A50000303C04A60000303D0400
:10460000A700B7319527A23141012508C30024082E
:10461000C20035084302031D0F2B34084202031861
:10462000122B132B152B0030BA2B4608B600B701FE
:10463000B635B70DB635B70DB635B70DB635B70DBE
:10464000B635B70D3608083EB8000030373DB90022
:104650003808BA003908BB000030BB1BFF30BC0073
:10466000BD0000303A04A40024303B04A500003013
:104670003C04A60000303D04A700B7319527A231C5
:1046800041012508C5002408C4004408B6004508B7
:10469000B700B801B9010830B635B70DB80DB90D7E
:1046A000890B4C2B4608BA00BB01BA35BB0DBA3595
:1046B000BB0DBA35BB0DBA35BB0DBA35BB0D3A08CB
:1046C000103EBC0000303B3DBD003C08BE003D0834
:1046D000BF000030BF1BFF30C000C10036083E04E1
:1046E000A40037083F04A50038084004A600390894
:1046F0004104A7003308A9003208A8003508AB0020
:104700003408AA00A0310120A23141013408C407B5
:104710003508C53D4608B600B701B635B70DB63504
:10472000B70DB635B70DB635B70DB635B70D36087A
:10473000083EB8000030373DB9003808BA003908E3
:10474000BB000030BB1BFF30BC00BD0000303A0492
:10475000A40024303B04A50000303C04A600003037
:104760003D04A7004508A9004408A800B43111245D
:10477000A231013008004001C2004208B200B3017A
:10478000B235B30DB235B30DB235B30DB235B30D8D
:10479000B235B30D3208083EB4000030333DB500E9
:1047A0003408B6003508B7000030B71BFF30B8003A
:1047B000B90000303604F40026303704F50000302C
:1047C0003804F60000303904F700B631D726A3319B
:1047D00075084001BF007408BE0031083F02031D88
:1047E000F32B30083E020318F62BF72BFB2B3F0868
:1047F000B1003E08B00030083104031D002C012C2C
:10480000042CAE01AF01B32C4208B200B301B235A3
:10481000B30DB235B30DB235B30DB235B30DB235FC
:10482000B30D3208083EB4000030333DB500340803
:10483000B6003508B7000030B71BFF30B800B9002C
:1048400000303604F40028303704F5000030380416
:10485000F60000303904F700B631D726A3317508C9
:104860004001C1007408C0002E082F040319392C20
:104870003A2C7A2C4008B2004108B300B401B501CB
:104880000830B235B30DB40DB50D890B412C42087B
:10489000B600B701B635B70DB635B70DB635B70D9D
:1048A000B635B70DB635B70D3608183EB80000302E
:1048B000373DB9003808BA003908BB000030BB1BCF
:1048C000FF30BC00BD0032083A04F40033083B045A
:1048D000F50034083C04F60035083D04F7002F08C5
:1048E000F9002E08F8003108FB003008FA00B33157
:1048F0004F23A33140013008C0073108C13D4208B1
:10490000B200B301B235B30DB235B30DB235B30D4C
:10491000B235B30DB235B30D3208083EB4000030E5
:10492000333DB5003408B6003508B7000030B71B7A
:10493000FF30B800B90000303604F40028303704E6
:10494000F50000303804F60000303904F700410863
:10495000F9004008F800B3311623A33140013108B3
:10496000AF003008AE0008004101C6004608B6009E
:10497000B701B635B70DB635B70DB635B70DB63587
:10498000B70DB635B70D3608083EB8000030373DD4
:10499000B9003808BA003908BB000030BB1BFF3033
:1049A000BC00BD0000303A04A40026303B04A50042
:1049B00000303C04A60000303D04A700B731952725
:1049C000A43141012508C3002408C2003508430270
:1049D000031DEC2C340842020318EF2CF02CF42CAD
:1049E0004308B5004208B40034083504031DF92C0F
:1049F000FA2CFD2CB201B301AC2D4608B600B7016C
:104A0000B635B70DB635B70DB635B70DB635B70DEA
:104A1000B635B70D3608083EB8000030373DB9004E
:104A20003808BA003908BB000030BB1BFF30BC009F
:104A3000BD0000303A04A40028303B04A50000303B
:104A40003C04A60000303D04A700B7319527A431EF
:104A500041012508C5002408C400320833040319A5
:104A6000322D332D732D4408B6004508B700B80128
:104A7000B9010830B635B70DB80DB90D890B3A2D0F
:104A80004608BA00BB01BA35BB0DBA35BB0DBA3505
:104A9000BB0DBA35BB0DBA35BB0D3A08183EBC008C
:104AA00000303B3DBD003C08BE003D08BF0000306B
:104AB000BF1BFF30C000C10036083E04A400370809
:104AC0003F04A50038084004A60039084104A700A7
:104AD0003308A9003208A8003508AB003408AA0042
:104AE000B4315524A43141013408C4073508C53D0B
:104AF0004608B600B701B635B70DB635B70DB635B1
:104B0000B70DB635B70DB635B70D3608083EB80047
:104B10000030373DB9003808BA003908BB00003012
:104B2000BB1BFF30BC00BD0000303A04A40028309D
:104B30003B04A50000303C04A60000303D04A70063
:104B40004508A9004408A800B4311124A43141014A
:104B50003508B3003408B200080000304101EE000F
:104B60006E084301D3000330460145054301BF00F1
:104B70003F030319BC2DBE2D0130BF2D0030BC00FA
:104B80000330460145054301BF0002303F060319CB
:104B9000CA2DCC2D0130CD2D0030BB004601AD011A
:104BA00043013B080319D52DD62DDF2D41016E0899
:104BB0000319DB2DDC2DDF2D4601AD01AD0A4601C9
:104BC0002D08031DE42DE62D0130E72D00304001B6
:104BD000E00046014508031DEE2DEF2DF82D2408B9
:104BE000031DF32DF52D0130F62D00304301BC00DF
:104BF000400194129A1243013C080319002E012E21
:104C0000102EB031D520A5310130B1317F21A53131
:104C10000130BD31A225A531B7313527A5315A2E36
:104C20003E080319142E152E3B2E40011813153083
:104C30004301C0004B30BF00BE30890B1D2EBF0B9F
:104C40001D2EC00B1D2E000040011817053043011A
:104C5000C0000F30BF00F130890B2C2EBF0B2C2E63
:104C6000C00B2C2E43013B080319372E382E3B2E48
:104C7000B431E624A53141016E08031D402E412EBA
:104C8000482EBE313C26A531BE31A726A5315A2E6D
:104C9000B031D520A531B031AD20A5314301530845
:104CA0000319532E542E5A2E42019E1244309B005B
:104CB0009C019E16A8304101A0002D30A100BD31FD
:104CC0002925A531BC31A924A53109304301C000F3
:104CD0001E30BF00E430890B6B2EBF0B6B2EC00B58
:104CE0006B2E000041016E080319772E782EA12E3D
:104CF0004601C30120304302031C7F2E802E812EEB
:104D0000BC2E0C304301C0009130BF000030890B35
:104D1000872EBF0B872EC00B872E0000460143084D
:104D20004301BF00C0013F084101A000430140080A
:104D30004101A100BF311927A53103144601C30D5C
:104D40007A2E0030A000A100BF311927A53109300B
:104D50004301C0001E30BF00E430890BAD2EBF0BF5
:104D6000AD2EC00BAD2E000001304101A00000307F
:104D7000A100BF311927A5314601C10143013C08FB
:104D80000319C42EA131F3298931EF294101CC0047
:104D9000FF30A0000030A1000430A2000030A300CA
:104DA0006C30AA314722A63100304101A000A10099
:104DB0000430A2000030A3006830AA314722A63197
:104DC00041014C08C400C501C435C50DC435C50D2D
:104DD000C435C50DC435C50DC435C50D4408083EE0
:104DE000C6000030453DC7004608C8004708C90056
:104DF0000030C91BFF30CA00CB0004304804A400B7
:104E00001F304904A50000304A04A60000304B04BE
:104E1000A7000230A800B3318E23A63141014C080F
:104E2000C400C501C435C50DC435C50DC435C50D97
:104E3000C435C50DC435C50D4408083EC600003054
:104E4000453DC7004608C8004708C9000030C91BD7
:104E5000FF30CA00CB0004304804A4001E304904CF
:104E6000A50000304A04A60000304B04A700023021
:104E7000A800B3318E23A63144304101B200003086
:104E8000B3006C30B4004330B5000030B6004C08BD
:104E900099310621A631B4319C24A631FF3041015D
:104EA0003605C4000F303705C5004408C600450864
:104EB000C7000030C71BFF30C800C90000304606DD
:104EC0004201DA005030410147064201DB00B030B8
:104ED000410148064201DC00AE3041014906420171
:104EE000DD005D084401D50042015C084401D400A6
:104EF00042015B084401D30042015A084401D20038
:104F0000410143084201E000410143080319892F90
:104F10008A2FA02F0030A000A1000430A200003092
:104F2000A3006C30AA314722A63101304201DE00D5
:104F30000030DF0004304301B2000030B300BD2F69
:104F40000030A7000030A6000F30A5000030A400FC
:104F50006C30A8000230A9000430AA000030AB0079
:104F6000B4315524A63108304201DE000030DF00A4
:104F700040304301B2000030B300FF304101A000D7
:104F80000030A1000430A2000030A3006430AA3138
:104F90004722A63100304101A000A1000430A20048
:104FA0000030A3006030AA314722A631003043010F
:104FB000AB000030AA000030A9000030A8002B0888
:104FC0004201D50043012A084201D40043012908C7
:104FD0004201D300430128084201D2005508D900FC
:104FE0005408D8005308D7005208D60000304401B6
:104FF000D1000030D0000030CF000030CE000800DB
:105000004101A400BC31DF24A831003A031909286A
:105010000A280F2854011F1B0E280F281428BE3100
:10502000BD26A83100301A2841012408BD31D625FB
:10503000A83101300800400194119A110530430154
:10504000C0000F30BF00F130890B2428BF0B24288B
:10505000C00B2428031040010E1E03140030031857
:1050600001304301BB003B08031937283828432887
:105070003E0803193C283D283F28D0014328410120
:105080006E084001E00000304101A0000030A100A6
:105090000130A200B131AE21A831B0311A20A831BF
:1050A000410121081F394601A400B0311A20A8315E
:1050B000410121084601C50045083F394301D2009E
:1050C000B0311A20A831410121084601C500450828
:1050D00020394301D1004601451D6F287128013058
:1050E000722800304301BD003D08031D782879284F
:1050F000952841016E0803197E288028A531F82DD6
:1051000043013C08031D852886287E283B08031D93
:105110008A288B287E283E0803198F2890289528F6
:105120005308031D942895287E2846014508033915
:10513000031D9C28A531AD2D0130A531AE2DAB301E
:1051400040012206031DA528A728983126280230F1
:105150002302031CAC28AD28A52808302102031C1B
:10516000B228B328A528263601394301BF00C00163
:10517000400124084301C1000230C136890BBD281B
:1051800041080639C200C301400125081F39430107
:10519000C400C501C435C50DC435C50DC435C50D24
:1051A00040012508C0394301C600C701C635C70DF7
:1051B000C635C70D44084604C80045084704C90061
:1051C00042084804CA0043084904CB003F084A0487
:1051D000B40040084B04B500F7303405BF0003307D
:1051E0003505C000E7303F064004031DF828F928C4
:1051F000FF280130B4000030B500983164286E30CB
:105200003405BF0000303505C00066303F0640045D
:10521000031D0B290C2911290230B4000030B50000
:10522000FD28B41B142915291A290330B4000030B5
:10523000B500FD28341B1D291F2998310128043091
:10524000B4000030B500FD28FC3041019E053F3020
:10525000BF313227A93100304101CE000030CD00EE
:105260000030CC000030CB00CF01D0010D30890BD5
:1052700037290000BC31AC24A931BC31E624A93166
:10528000003A0319442945293D29BC31BF24A931DD
:1052900041012008CB072108CC3D0030CD3DCE3D5B
:1052A0000130CF070030D03D5008803AC600803032
:1052B0004602031D5D290A304F02031C6029612943
:1052C0003629033041019E040030B9000030B80097
:1052D0000030B7000A30B600430123084101AD0099
:1052E000430122084101AC00430121084101AB0008
:1052F000430120084101AA000030B1000030B00095
:105300000330AF00FF30AE00B2314022A93141017D
:105310002D08BD002C08BC002B08BB002A08BA00D1
:10532000B6317C26A93141013908CA003808C900C4
:105330003708C8003608C7004E08B9004D08B80045
:105340004C08B7004B08B6004A08BD004908BC002D
:105350004808BB004708BA00B6317C26A931410194
:105360003708C5003608C4000800F80154011D1DA7
:10537000BA29BB29BD2940015E1454019D1CC129D5
:10538000C229C8291D121D164001DE14F801F80AB1
:1053900054011908FA0078080319CF29D029D42913
:1053A000BE311226A931462A41016E08031DD929B2
:1053B000DA29E1297A08F4000130AC313224A9312C
:1053C000462A40016203031DE629E7291E2AAA3066
:1053D0007A06031DEC29ED291E2A3F3043015202B3
:1053E000031CF329F429FC29E43000320032890B34
:1053F000F529003200320A2A5208F9007908031D03
:10540000022A032A042A0A2A1830890B052A0130A5
:10541000F902FE2940016108BF310027A931003A95
:105420000319132A142A462A02304001E2007A089E
:10543000F4000130AC313224A931462A0230620630
:10544000031D232A242A402A7A086106031D292ADB
:105450002A2A312A7A08F4000230AC313224A931E8
:10546000372A7A08F4000A30AC313224A9314001DD
:10547000E2010030F000F100BE317B26A931462A5E
:105480007A08F4000130AC313224A931080041011E
:10549000A8002808A90022082304031D502A512A25
:1054A000522AE02A2908860002308700200881005D
:1054B00022082907A4002408FF3E86000230870046
:1054C0002008810000302302033003192202031850
:1054D0006A2A6B2A6C2AE02A290A86000230870091
:1054E000200881002908023E86000230870020083B
:1054F000810022082907A4002408FE3E860002300D
:1055000087002008810022082907A4002408FD3E06
:105510008600023087002008810000302302073017
:10552000031922020318952A962A972AE02A2908A5
:10553000033E8600023087002008810022082907E8
:10554000A4002408FC3E8600023087002008810069
:10555000003023020930031922020318B02AB12AAD
:10556000B22AE02A2909A4002A09A500A40A0319DD
:10557000A50A03302405A60000302505A70026084B
:10558000A4002408A9072608A2022708A33BFC3090
:10559000A205FF30A305DA2A290886000230870019
:1055A000200881000130A2020030A33B0130A4009A
:1055B0002408A90722082304031DDF2AE02ACC2A95
:1055C00008003C30BF313227AA3100304101D500FC
:1055D0000030D4000030D3000030D200D601D70113
:1055E0000D30890BF12A0000BC31AC24AA3187317F
:1055F000F827AA31BC31E624AA31003A0319012B5D
:10560000022BFA2ABC31BF24AA3141012008D2075B
:105610002108D33D0030D43DD53D0130D6070030C0
:10562000D73D5708803AC60080304602031D1A2B2A
:105630000A305602031C1D2B1E2BF02A4301300892
:105640004101C600430131084101C700C801C90139
:105650005208CA005308CB005408CC005508CD00AE
:105660000130CA35CB0DCC0DCD0D890B312B460841
:10567000CA024708CB3B4808CC3B4908CD3B4D0804
:10568000AD004C08AC004B08AB004A08AA0043012F
:1056900023084101B100430122084101B000430148
:1056A00021084101AF00430120084101AE00B231A1
:1056B0004022AA3141012D08D1002C08D0002B082E
:1056C000CF002A08CE000030B9003930B800813050
:1056D000B7009C30B6005108BD005008BC004F0810
:1056E000BB004E08BA00B6317C26AA315A304101BF
:1056F000C60036084602C40037090318890AC500E7
:1057000008004001EB00F02B40016B084101B300A1
:10571000B401B335B40DB335B40DB335B40DB335F1
:10572000B40DB335B40D3308083EB5000030343D38
:10573000B6003508B7003608B8000030B81BFF3097
:10574000B900BA0000303704AD0001303804AE00B3
:1057500000303904AF0000303A04B0000230B1002C
:10576000B0313C20AB31302C32080319B82BB92BA7
:10577000EE2B40016B084101B300B401B335B40D09
:10578000B335B40DB335B40DB335B40DB335B40D75
:105790003308083EB5000030343DB6003508B70088
:1057A0003608B8000030B81BFF30B900BA0000302E
:1057B0003704A4000C303804A50000303904A600DA
:1057C00000303A04A7003208A8000030A9000430D5
:1057D000AA000030AB00B4315524AB310130312C7C
:1057E0006B084101B300B401B335B40DB335B40D4A
:1057F000B335B40DB335B40DB335B40D3308083E2D
:10580000B5000030343DB6003508B7003608B800A2
:105810000030B81BFF30B900BA0000303704A400D4
:1058200003303804A50000303904A60000303A04E3
:10583000A700A801B3318E23AB314101BB00BC01ED
:105840003C08003A0319252C302C3B08133A031965
:10585000842B073A0319302C033A0319B42B302C4C
:1058600000300800F70043013C080319382C392C9C
:10587000862C65305402031C3E2C3F2C442CBE3138
:105880001226AC310030E52C41016E080319492C79
:105890004A2C552C7703031D4E2C4F2C612C803045
:1058A00074020318542C552C612C430154088600B3
:1058B00003308700740881000130F5007508D407B3
:1058C000842C430154088600033087007408F500D7
:1058D0000630F536890B692C7708F6000130F6356D
:1058E000FF3E031D6F2C76357504C03881000130F2
:1058F000F5007508D4075408860003308700740843
:105900003F39803881005C2C0130E52C3E080319BA
:105910008A2C8B2C9B2C3B0803198F2C902C9B2CB6
:1059200050080319942C952C422C40018D1C992C65
:105930009A2C9B2C422CBC31D824AC31003A031950
:10594000A22CA32CA92C420163080319A82CA92C72
:10595000AC2C4E0119163F2C41016E080319B12CD5
:10596000B22CC32C7703031DB62CB72CC82C4001D6
:105970006008031DBC2CBD2CC82C80307402031899
:10598000C22CC32CC82C7408BD314F25AC31842CDB
:105990007408F5000630F536890BCB2C7708F60035
:1059A0000130F635FF3E031DD12C76357504C03825
:1059B000BD314F25AC3174083F3980384201E400D5
:1059C000E301E30A4E011916842C08004001D301BB
:1059D00043013C080319ED2CEE2C032D54304001FB
:1059E000C3000030C4000130C5000030C6000130E3
:1059F000B5313225AC314001430344040319012D74
:105A0000022D192DA72D42011D1D072D082D0A2D30
:105A100040015E1642019D1C0E2D0F2D152D1D12ED
:105A20001D164001DE16D301D30A420119084001B8
:105A3000D400530803191D2D1E2D222DBE31122610
:105A4000AC31A72D41016E08031D272D282D952D62
:105A500040015408BF310027AC31A72D6308D000A6
:105A60000230D036890B312D50080F39D2003F302B
:105A70005405D00063080339D1000530D135FF3E0D
:105A8000031D3E2D51355004D4006A2D5408EA0000
:105A9000E301E201DF01DF0A802D5408BF31002756
:105AA000AC31802D5408E100AA306106031D592D48
:105AB0005A2D5C2DE201802DE201E20A0130F00056
:105AC0000030F100BE317B26AC31802D5408E90056
:105AD000DD01802D5208D000D1015108003A031990
:105AE000722D802D5008003A0319462D013A0319F2
:105AF0004D2D033A0319522D013A0319662D802DBD
:105B00004001E301A72D5408E300A72D6008031905
:105B10008A2D8B2D902D5E16BE311226AC31802D34
:105B20005408BF310027AC31802D40015408C039E2
:105B3000D000D1015108003A03199F2D862D50083D
:105B4000803A03192E2D403A0319832D862D080023
:105B50000130F80078084301BA070A303A02031C02
:105B6000B22DB32D6B2EBA010130AC070030AD3D24
:105B70000030AE3D0030AF3DBE2D6B2E40015F08C2
:105B80000319C32DC42DF32D023043012C07CC0083
:105B900000302D3DCD0000302E3DCE0000302F3D99
:105BA000CF0041016E080319D62DD72DF02D4001ED
:105BB0006A080139F4000030AC313224AD313230A2
:105BC000F0000030F100BE317B26AD3102304001E3
:105BD0005F02031CEC2DED2DF02DBE319126AD3171
:105BE0004001DF01112E43014F082F02031D022E39
:105BF0004E082E02031D022E4D082D02031D022EFB
:105C00004C082C02031C052E062E112E0030CF004E
:105C10000030CE000030CD000030CC00BE31272651
:105C2000AD3141016E080319162E172E6B2E40015F
:105C30005E0803191C2E1D2E6B2E43013C08031D0C
:105C4000222E232E312EBC31D824AD31003A031937
:105C50002A2E2B2E6B2E42016308031D302E312E6F
:105C60006B2E40015E1C352E362E402EFE30F80085
:105C70007808DE05F4010B30AC313224AD316B2EE7
:105C8000DE1C432E442E4F2EFD30F8007808DE0532
:105C9000F401F40A0B30AC313224AD316B2E5E1EB0
:105CA000522E532E5D2EEF30F8007808DE05F401F9
:105CB0000C30AC313224AD316B2EDE1E602E612EE5
:105CC000BD2DDF30F8007808DE05F401F40A0C3051
:105CD000AC313224AD31080082302506031D712E0F
:105CE000722E7E2E53302606031D772E782E7E2EA2
:105CF0006330270603197D2E7E2E8B2E410164080A
:105D00006202D3006508633BD4006608BD31FE25FE
:105D1000AE319031D1284101DB01FF3042015E05F7
:105D2000A00000305F05A100033020062104031D00
:105D30009A2E9C2E8F311A2F00304301AB00003079
:105D4000AA000030A9000030A8002B084201D500AD
:105D500043012A084201D400430129084201D3002B
:105D6000430128084201D2009A2EA430C700023015
:105D7000C8000130C9000030CA006608B531D3251B
:105D8000AE31410147084804031DC72EC82ECA2E54
:105D90008F31262F0130E4070030E53D450124080E
:105DA0004101E000600A031DD62ED72ED82EC82E42
:105DB0006008031DDC2EDD2EDE2E9A2EA430C700D7
:105DC0000230C8000130C9000030CA006608B53191
:105DD000D325AE31410147084804031DF02EF12EB2
:105DE000F22EC82E0130E4070030E53D45012408BD
:105DF0004101E10061080319FE2EFF2E262FA43079
:105E0000C7000230C80061084201A000A1012008BB
:105E10004101C900420121084101CA006608B531AB
:105E2000D325AE31410161084201A200A301410125
:105E3000480842012306031D212F41014708420162
:105E400022060319242F252F262FC82E4101610871
:105E50004201A000A10120084101E40742012108FC
:105E60004101E53D8E31FA2E0230BF313227AF318C
:105E7000FF304101CD00FF30CE00CF01D001CB017A
:105E8000CC01BC31AC24AF31BC31E624AF31003A97
:105E900003194B2F4C2F442FBC31BF24AF3141018C
:105EA0002108D2002008D1004E085202031D5A2FAB
:105EB0004D08510203185D2F5E2F622F5208CE004D
:105EC0005108CD0052085002031D682F51084F029F
:105ED00003186B2F6C2F702F5208D0005108CF0081
:105EE0000130CB070030CC3D4C08803AC6009230E0
:105EF0004602031D7D2F1C304B02031C802F812F77
:105F0000412F00304101B9000D30B800B130B70069
:105F10005830B6004D08AA004E08AB00AC01AD01E8
:105F2000430123084101B100430122084101B000AF
:105F3000430121084101AF00430120084101AE00A7
:105F4000B2314022AF3141012D08BD002C08BC0008
:105F50002B08BB002A08BA00B6317C26AF314101BC
:105F600036080B3ECD000030373DCE000030B90082
:105F70000D30B800B130B7005830B6004F08AA0055
:105F80005008AB00AC01AD01430123084101B10051
:105F9000430122084101B000430121084101AF0043
:105FA000430120084101AE00B2314022AF3141012E
:105FB0002D08BD002C08BC002B08BB002A08BA0025
:105FC000B6317C26AF31410136080B3ECF000030A0
:105FD000373DD000FF304D05C60000304E05C700EC
:105FE000FF304F05C80000305005C9004808C900FF
:105FF000C80146084804C40047084904C500080011
:1060000041012108A3002008A2000A280130A007AE
:106010000030A13D20088400210885001200031DE6
:1060200012281328062822082002A0002308213B5A
:10603000A100080050011E140000000050011D08BE
:106040004101A30050011C084101A20001304001A0
:10605000EB006B0850019A07031D2F2830283628C3
:1060600001304001EB006B0850019B074101230800
:10607000A1002208A0000800043041012D04A40062
:1060800000302E04A50000302F04A600003030049C
:10609000A7003108A800B3318E23B0314101300888
:1060A000A7002F08A6002E08A5002D08A400A8010F
:1060B000B3318E23B031003A031D5F2860284E288B
:1060C000080040015D0803196628672886281130FA
:1060D0004201620203186D286E28862862083D3E40
:1060E0008600023087000108F4000330AC3132240E
:1060F000B031003A03197D287E2886280130F80047
:1061000078084201E20701304001DD020800A028C2
:106110007008860071088700010843018C004E0159
:106120000F1C932894288F280F1070088600710880
:10613000870043010C0881000130F0070030F13D79
:106140000130F2020030F33B720A031DAB28730AE0
:10615000031DAB28AC28882808000F307E019B0067
:106160000A307D01CB004E019912A0304101A00000
:106170003C30A100BC31FC24B0314E011912A630D4
:106180004101A0003C30A100BD310525B0310830EF
:1061900042019F0090309D0024309E0040309B00C3
:1061A00003309C004E019916080011307E01A100B9
:1061B00010307D01CD004E0199139E304101A000A9
:1061C0003C30A100BD310E25B0314E011913A33072
:1061D0004101A0003C30A100BD311725B03118307D
:1061E00054019F0090309D0024309E0004309B009D
:1061F0000D309C004E0199170800182920088600D0
:1062000021088700010843018C004E010F1C092959
:106210000A2905290F10410120088600210887005E
:1062200043010C08810001304101A0070030A13D6D
:1062300001304101A2020030A33B220A031D2429A0
:10624000230A031D24292529FE28080041012308CB
:10625000AA002208A9002108A8002008A7004429B4
:10626000290886002A0887000108A6000130A9072E
:106270000030AA3D270886002808870026088100EC
:106280000130A7070030A83D0130A4020030A53B33
:10629000240A031D4F29250A031D4F29502930299F
:1062A0000800403040019800203099009A014430A5
:1062B0009200C63093007D3094007E01CE01C30170
:1062C0000C30B800E501FF30C4004030B9007F3029
:1062D000CF00BA01C501D001FF30BB00FF30C600BE
:1062E000FF30D100FF30BC00FF30C700FF30D200CC
:1062F0000830E8000B30980013309300080040018C
:10630000EB004301901240016B0803198829892989
:10631000A4290C307D01C50015307E019C0043127C
:10632000400113127E01441616309B00C311400138
:1063300093117E01C4150A307D01C6007E01431110
:10634000400113157E014415403043018F00013098
:106350009000910101308D00901608004101200845
:10636000A3002108A4002208A5001030A536A40C23
:10637000A30C890BB62923080139A600A60EA60D89
:10638000A60D50011E0841012606BF392606500100
:106390009E0041012008A3002108A4002208A500B6
:1063A0000830A536A40CA30C890BD1292308500171
:1063B0009B004101200850019A0008004001EB00B9
:1063C0006B084101B200B301B235B30DB235B30D64
:1063D000B235B30DB235B30DB235B30D3208083E48
:1063E000B4000030333DB5003408B6003508B700BE
:1063F0000030B71BFF30B800B90000303604AD00E4
:1064000001303704AE0000303804AF0000303904EA
:10641000B0001030B100B0313C20B1310800400173
:10642000EB006B084101B200B301B235B30DB235D8
:10643000B30DB235B30DB235B30DB235B30D32086D
:10644000083EB4000030333DB5003408B6003508CE
:10645000B7000030B71BFF30B800B9000030360479
:10646000AD0001303704AE0000303804AF0000301A
:106470003904B0000830B100B0313C20B23108001E
:1064800000304101B5000030B4000030B3000030EE
:10649000B2002A1C4C2A4D2A552A2E08B2072F0872
:1064A000B33D3008B43D3108B53D0130AE35AF0DD8
:1064B000B00DB10D890B562A0130AD36AC0CAB0CCA
:1064C000AA0C890B5D2A2D082C042B042A04031D19
:1064D0006A2A6B2A492A3508AD003408AC00330813
:1064E000AB003208AA0008004001EB006B08410134
:1064F000B400B501B435B50DB435B50DB435B50D31
:10650000B435B50DB435B50D3408083EB6000030CD
:10651000353DB7003608B8003708B9000030B91B60
:10652000FF30BA00BB0000303804A4002630390424
:10653000A50000303A04A60000303B04A700B731A4
:106540009527B23141012508B3002408B2000800A4
:10655000400199127408F9007508FA007608FB00EA
:106560007708FC001030FC36FB0CFA0CF90C890B98
:10657000B32A7908E4007408F9007508FA0076086F
:10658000FB007708FC000830FC36FB0CFA0CF90C19
:10659000890BC42A7908E5007408E6007808E7004A
:1065A0006430F0000030F1000430F2000030F300FD
:1065B000B0318720B2314001991608004001EB004C
:1065C0006B084101AD00AE01AD35AE0DAD35AE0D80
:1065D000AD35AE0DAD35AE0DAD35AE0D2D08083E69
:1065E000AF0000302E3DB0002F08B1003008B200DF
:1065F0000030B21BFF30B300B40000303104A400FF
:1066000002303204A50000303304A6000030340408
:10661000A700A801B3318E23B2310A390319112B17
:10662000122B142B0130152B003008004001991259
:106630007408FA007508FB007608FC007708FD0076
:106640001030FD36FC0CFB0CFA0C890B212B7A0860
:10665000E4007408FA007508FB007608FC0077086F
:10666000FD000830FD36FC0CFB0CFA0C890B322BBC
:106670007A08E50074080438E6007908E70078082D
:10668000E8006430F0000030F1000530F200003026
:10669000F300B0318720B331400199160800400162
:1066A00099127408A9007508AA007608AB0077084B
:1066B000AC001030AC36AB0CAA0CA90C890B5A2BD1
:1066C0002908E4007408A9007508AA007608AB0040
:1066D0007708AC000830AC36AB0CAA0CA90C890BBF
:1066E0006B2B2908E5007408E6006430F0000030E8
:1066F000F1000330F2000030F300B0318720B331F5
:106700007908F1007808F0007B08F3007A08F200BD
:10671000B0318720B3314001991608004001991229
:1067200041012408A9002508AA002608AB00270873
:10673000AC001030AC36AB0CAA0CA90C890B9A2B10
:1067400029084001E40041012408A9002508AA0005
:106750002608AB002708AC000830AC36AB0CAA0CFE
:10676000A90C890BAD2B29084001E5004101240843
:106770004001E600410128084001E7006430410182
:10678000A0000030A1000430A2000030A300B0310E
:10679000FD20B33140019916670808004101A300AC
:1067A0002308A4002008A500E52B0130A102003039
:1067B000A23B01304001EB006B084101A40701300E
:1067C0004001EB006B084101A507210822040319D1
:1067D000EA2BEB2BF92B25088600023087002408D2
:1067E000840002308500000801060319F82BF92BFC
:1067F000D52B21082204031DFE2BFF2B022CA00108
:10680000A101102C2408860002308700250884008E
:106810000230850000080102A000A101031CA103B1
:1068200008004001991241012408AA002508AB0084
:106830002608AC002708AD001030AD36AC0CAB0C10
:10684000AA0C890B1D2C2A084001E40041012408F0
:10685000AA002508AB002608AC002708AD000830C8
:10686000AD36AC0CAB0CAA0C890B302C2A084001BD
:10687000E5004101240804384001E60041012908EF
:106880004001E700410128084001E800643041016F
:10689000A0000030A1000530A2000030A300B031FC
:1068A000FD20B431400199160800400199124101C0
:1068B0002408AC002508AD002608AE002708AF006C
:1068C0001030AF36AE0CAD0CAC0C890B612C2C0823
:1068D0004001E40041012408AC002508AD00260871
:1068E000AE002708AF000830AF36AE0CAD0CAC0CD4
:1068F000890B742C2C084001E5004101240840015B
:10690000E60064304101A0000030A1000330A20085
:106910000030A300B031FD20B43141012908A100AD
:106920002808A0002B08A3002A08A200B031FD20EF
:10693000B43140019916080044015F084101AD00DF
:1069400044015E084101AC0044015D084101AB0017
:1069500044015C084101AA004C30B1009530B00000
:106960007F30AF002D30AE00B2314022B431013063
:1069700041012A074401DC00003041012B3D440164
:10698000DD00003041012C3D4401DE0000304101BA
:106990002D3D4401DF005C084101B80044015D0861
:1069A0004101B90044015E084101BA0044015F0899
:1069B0004101BB001130BB36BA0CB90CB80C890BC5
:1069C000DB2C3908B7003808B6000800430150082E
:1069D0000319EB2CEC2CF32C40018D1CF02CF12C2A
:1069E000F32C4301D00143015008031DF82CF92C6E
:1069F000312D292D32304101A0000030A100BF31DE
:106A00001927B43101309231E622B4310530410109
:106A1000EB000F30EA00F130890B0C2DEA0B0C2D46
:106A2000EB0B0C2D00304101A000A100BF31192754
:106A3000B43101309231E622B43105304101EB002E
:106A40000F30EA00F130890B232DEA0B232DEB0BDD
:106A5000232D40018D182D2D2E2DFA2C4301D00110
:106A6000D00A08004001CF004408AF004308AE0040
:106A70004608B1004508B0004F08A331BB23B5312B
:106A800040012F08C6002E08C50045084604031D16
:106A90004A2D4B2D4E2DC301C401802D4F08C70038
:106AA000C801C735C80DC735C80DC735C80DC735AE
:106AB000C80DC735C80D4708083EC9000030483D1D
:106AC000CA004908CB004A08CC000030CC1BFF307C
:106AD000CD00CE0004304B04F40001304C04F5002E
:106AE00000304D04F60000304E04F7004030F8004E
:106AF000B231A822B53140014608C4004508C300A0
:106B0000080000304101A0000030A1000030A200C8
:106B1000B131AE21B5314401D601D7014101A70100
:106B2000A801B0311A20B531410120084401D6072F
:106B3000410121084401D73D01304101A707003040
:106B4000A83D04302802003003192702031CA92D98
:106B5000AA2D912D0030A0000430A1000030A20029
:106B6000B131AE21B5314401D801D9014101A901AA
:106B7000AA01B0311A20B531410120084401D807DB
:106B8000410121084401D93D01304101A9070030EC
:106B9000AA3D3C302A02003003192902031CD12DE2
:106BA000D22DB92D08004001EB0041014808B30087
:106BB0004708B2004A08B5004908B40040016B0814
:106BC000A431B424B53141013308CA003208C900E8
:106BD00049084A04031DED2DEE2DF12DC701C80112
:106BE000252E40016B084101CB00CC01CB35CC0DEB
:106BF000CB35CC0DCB35CC0DCB35CC0DCB35CC0D31
:106C00004B08083ECD0000304C3DCE004D08CF0073
:106C10004E08D0000030D01BFF30D100D20004302D
:106C20004F04A40001305004A50000305104A60018
:106C300000305204A7004030A800B3318E23B53194
:106C400041014A08C8004908C70008001630410140
:106C5000A7000130A8000130A900BD31C325B6311D
:106C600041012808AB002708AA000A30AC00003018
:106C7000AD00BF319F27B63141012B084301B10060
:106C800041012A084301B00019304101A700013039
:106C9000A8000130A900BD31C325B6314101270844
:106CA000B6002808B700B801B9013908AD003808A6
:106CB000AC003708AB003608AA000030B100003045
:106CC000B0000030AF006430AE00B2314022B631C7
:106CD00041012D084301A30041012C084301A200FA
:106CE00041012B084301A10041012A084301A000F2
:106CF000B5318125B631080000304101C2000030B5
:106D0000C1000030C0000030BF003908380437042B
:106D1000360403198C2E8D2ECE2EC301C30A9B2E52
:106D20000130B635B70DB80DB90D890B912E013074
:106D3000BE003E08C307B91F9E2E9F2E902E013025
:106D4000BF35C00DC10DC20D890BA02E39083D0203
:106D5000031DB42E38083C02031DB42E37083B0235
:106D6000031DB42E36083A02031CB72EB82EC12ECE
:106D70003608BA023708BB3B3808BC3B3908BD3B74
:106D80003F140130B936B80CB70CB60C890BC22EC3
:106D90000130C302031DCD2ECE2E9F2E4208B90016
:106DA0004108B8004008B7003F08B600080040019D
:106DB000AB01AB0A99127408F8007508F90076085F
:106DC000FA007708FB001030FB36FA0CF90CF80CCF
:106DD000890BE42E7808E4007408F8007508F900BF
:106DE0007608FA007708FB000830FB36FA0CF90C3D
:106DF000F80C890BF52E7808E5007408E60064307D
:106E0000F0000030F1000530F2000030F300B03146
:106E10008720B631400199162D08AA002C08A90038
:106E20006808F800F9016708FA00FB017A08FB001E
:106E3000FA0178087A04AC0079087B04AD002B08CD
:106E40000319232F242F262FAB01DA2E2A082D0613
:106E5000031D2C2F29082C06031D2F2F302FDA2E6F
:106E60002D08F5002C08F4000800420165080319FC
:106E70003A2F3B2F4A2F15304101AE004B30AD0069
:106E8000BE30890B412FAD0B412FAE0B412F0000BF
:106E90004201E50100304101A7000030A6000030AA
:106EA000A5000430A4008030A800B3318E23B73190
:106EB00009304101AE001E30AD00E430890B5E2F79
:106EC000AD0B5E2FAE0B5E2F00000A304101AF000C
:106ED0000030B000822F01304101AF020030B03BE2
:106EE0002F0A031D772F300A031D772F782F792F54
:106EF000942FD0304101AD00C930890B7D2FAD0BEF
:106F00007D2F003200304101A7000030A600003084
:106F1000A5000030A400A801B3318E23B731803919
:106F2000031D932F942F6B2F08004101AF01AF0A6F
:106F30004001991241012408A8002508A90026084B
:106F4000AA002708AB001030AB36AA0CA90CA80C7D
:106F5000890BA42F28084001E40041012408A8005F
:106F60002508A9002608AA002708AB000830AB3680
:106F7000AA0CA90CA80C890BB72F28084001E50022
:106F8000410124084001E60064304101A0000030C6
:106F9000A1000530A2000030A300B031FD20B731C0
:106FA0004001991641013108AE003008AD004001A2
:106FB00068084101A800A901400167084101AA0031
:106FC000AB012A08AB00AA0128082A04B00029084E
:106FD0002B04B1002F080319EE2FEF2FF12FAF0173
:106FE000982F2E083106031DF72F2D083006031D9C
:106FF000FA2FFB2F982F3108A5003008A4000800B5
:1070000000340034003400340034003400340034E0
:1070100000340034003400340034003400340034D0
:1070200000340034003400340034003400340034C0
:1070300000340034003400340034003400340034B0
:0E704000613465346234753473343334003493
:10793C00080008000800FF3401344E011913080038
:10794C004E01191208004B019E17080041019D14AD
:10795C000800BB3052018C000800803046019600B4
:10796C00950194010800163050018C0037308D00C1
:10797C00080041011C08A1001B08A00008006400BD
:10798C0080010131890BC62C0034FE0012001E0050
:10799C00FE0BCC2C003403104E01191F03140030C5
:1079AC00093D080003104E01191E03140030093D57
:1079BC00080003104E01191F03140030093D080084
:1079CC00031041019D1C03140030093D08000310F5
:1079DC004E01191E03140030093D0800823053017A
:1079EC00900091010630920093010800410121089A
:1079FC004001D800410120084001D7000800410196
:107A0C0021084001D600410120084001D5000800A2
:107A1C00410121084001DC00410120084001DB004C
:107A2C000800410121084001DA0041012008400111
:107A3C00D9000800A33041019E009F019B019C01CD
:107A4C0001309D000800410121084301B9004101AA
:107A5C0020084301B800080001340034003400341D
:107A6C00013401343F3401344734603051018D000E
:107A7C008F01910106309300900192010800AE3401
:107A8C00B0345334EF34FE34EF34FF34FF34FF346E
:107A9C000034F0004E01191E542D552D562D19127F
:107AAC00700842019A004E0119160800430138086B
:107ABC0039040319622D632D682D39088A003808A2
:107ACC000A00BD3108004F01960102309700453085
:107ADC0098003330990001309A0006309B00080062
:107AEC0041012008FF3E4401DC00FF304101213DF3
:107AFC004401DD00DE01DF0108004001EB004E0116
:107B0C00191E892D8A2D8B2D191240016B084201EB
:107B1C009A004E01191608000130450190008F01A2
:107B2C0091010F308D008C014E019010FF304501FA
:107B3C008E000F308D0008004001EB006B0803191C
:107B4C00A82DA92DAF2D7E01C312400193127E01E9
:107B5C00C416400199160800F0004E01191FB72DEC
:107B6C00B82DB92D191354019E120D309C009E1680
:107B7C0070089A004E011917080041012708A0004F
:107B8C002808A1002908A200B131AE21BD31B031C5
:107B9C001A20BD3141012108A8002008A7000800C7
:107BAC004001EB004E01191FDC2DDD2DDE2D1913CC
:107BBC0054019E120D309C009E1640016B0854011E
:107BCC009A004E011917080001304301B235B30D6C
:107BDC00890BEC2D00303302413003193202031CA7
:107BEC00F82DF92DFD2D4030B2000030B300080007
:107BFC004101D5000030C7000030C8005408CA004D
:107C0C005308C9005508B531D325BD314101480889
:107C1C00D4004708D30008003230F0000030F100E7
:107C2C00BE317B26BE31053043012C07CC00003021
:107C3C002D3DCD0000302E3DCE0000302F3DCF002D
:107C4C00080041016E08031D2C2E2D2E352E0130FF
:107C5C00F0000030F100BE317B26BE313B2E0030EF
:107C6C00F000F100BE317B26BE31080010307D01E2
:107C7C00BB0003307E019B0002307C01A500A601F5
:107C8C00A701A801A9010230AA00AB01AC01AD010A
:107C9C008030A400080044304B019F00F9309D0057
:107CAC009C014E018C1296169F304101A0003C3075
:107CBC00A100BD312925BE3180304B019E0008004A
:107CCC0041016E08031D6B2E6C2E742E0130A0002A
:107CDC000030A100BF311927BE317A2E0030A00030
:107CEC00A100BF311927BE3108007108F3007008DC
:107CFC00F200F336F20CF336F20C720846019500E2
:107D0C0070080339F2000530F235FF3E031D8A2E50
:107D1C007235940008008B130B130530F1000F30F3
:107D2C00F000F130890B982EF00B982EF10B982E59
:107D3C0000007E019B01A10198019301A6010100A5
:107D4C0008000A307D01BD0004307E01A1008230A4
:107D5C007C01AF000230B000B101B201B3010230BE
:107D6C00B400B501B601B7018030AE000800323066
:107D7C004101A0000030A100BF311927BE310530F0
:107D8C0043012C07CC0000302D3DCD0000302E3DA2
:107D9C00CE0000302F3DCF0008008B130B130530A5
:107DAC004101A1000F30A000F130890BDB2EA00B9C
:107DBC00DB2EA10BDB2E7E019B01A101980193010F
:107DCC00A601010008004E018C1201304301B607D8
:107DDC000030B73D00303702C83003193602031C9F
:107DEC00F82EF92EFF2EBD315C25BE314301B601B4
:107DFC00B7010800F400BC31D124BF31003A03199B
:107E0C00082F092F0E2F54011F1B0D2F0E2F132F70
:107E1C00BE311226BF310030182F7408BD31B22587
:107E2C00BF310130080041012108A3002008A20045
:107E3C00A336A20CA336A20C2208460195004101E0
:107E4C0020080339A2000530A235FF3E031D2A2F5E
:107E5C0022354601940008004101A1001D0C890C3B
:107E6C003F39210603193B2F3C2F452F1D103B306A
:107E7C0088310020BF310D30890B422F00004101A9
:107E8C00210888310020BF3108004001EB006B084D
:107E9C00031D512F522F5B2F440159084101A100A2
:107EAC00440158084101A000632F440157084101C7
:107EBC00A100440156084101A000080042016308DA
:107ECC000319692F6A2F6E2F64089A00E3017F2F24
:107EDC004E01191241016E080319752F762F7F2F51
:107EEC0042016308031D7B2F7C2F7F2FB031612053
:107EFC00BF310800BD316925BF31B1315121BF31CE
:107F0C00BD313B25BF31BC31B924BF31BC31AF24AD
:107F1C00BF31BD319225BF31BE315126BF31BC318D
:107F2C00F424BF31BD312025BF31BC31B324BF3166
:107F3C0008004101AE01AF012A1CA52FA62FAA2FC4
:107F4C002C08AE072D08AF3D0130AC35AD0D890BBB
:107F5C00AB2F0130AB36AA0C890BB02F2A082B049F
:107F6C00031DB92FBA2FA22F2F08AB002E08AA0081
:107F7C0008004101A7002108A5002008A40027083B
:107F8C00A6002608860002308700A60A2508A30052
:107F9C002408A200A40A0319A50A220884002308B5
:107FAC0085000008C03F8908031DDD2FDE2FC72F79
:107FBC000800F22F200886002108870001084301E1
:107FCC008C0001304101A0070030A13D4E010F1C77
:107FDC00F02FF12FEC2F0F1001304101A2020030D5
:107FEC00A33B220A031DFE2F230A031DFE2FFF2F86
:047FFC00E02F08006A
:00000001FF
